:020000040000FA
:020000001B28BB
:08000800A200030E8312A10007
:100010000508A0000B108B1C11288B100230A01AB1
:100020000130A01D0130201E02308500210E83000A
:10003000A20E220E09008316FF2390009F01FC30C0
:1000400085001830960018308B000113831207309A
:100050009900023085009F018B172D2844342034ED
:100060005434793470346534203446346C34693413
:100070007034203446346C346F3470342E34203471
:100080005034653474346534203447347234693400
:100090006634663469347434683473342C342034F0
:1000A0004D346134793420343234303430343434A3
:0C00B0002E342034523431342E343234DB
:02400E00843FED
:00000001FF
